 returnadd

 Timestamp is 59c22125 (Wed Sep 20 16:04:53 2017)

 Preferred load address is 0000000000000000

 Start         Length     Name                   Class
 0001:00000000 0000136bH .text$mn                CODE
 0002:00000000 000006a8H .rdata                  DATA
 0002:000006a8 0000009cH .rdata$debug            DATA
 0003:00000000 00000000H .data                   DATA
 0003:00000000 00000020H .bss                    DATA
 0004:00000000 000000c0H .pdata                  DATA
 0005:00000000 0000008cH .xdata                  DATA

  Address         Publics by Value              Rva+Base               Lib:Object

 0000:00000000       __guard_fids_count         0000000000000000     <absolute>
 0000:00000000       __guard_flags              0000000000000000     <absolute>
 0000:00000000       __guard_fids_table         0000000000000000     <absolute>
 0001:00000000       _ModuleEntryPoint          00000000000002c0 f   UefiApplicationEntryPoint:ApplicationEntryPoint.obj
 0001:00000048       ProcessLibraryConstructorList 0000000000000308 f   returnadd:AutoGen.obj
 0001:000001ec       ProcessLibraryDestructorList 00000000000004ac f   returnadd:AutoGen.obj
 0001:000001f8       ProcessModuleEntryPointList 00000000000004b8 f   returnadd:AutoGen.obj
 0001:0000021c       UefiMain                   00000000000004dc f   returnadd:returnaddress.obj
 0001:00000258       DebugPrint                 0000000000000518 f   BaseDebugLibNull:DebugLib.obj
 0001:00000264       DebugAssert                0000000000000524 f   BaseDebugLibNull:DebugLib.obj
 0001:00000268       DebugAssertEnabled         0000000000000528 f   BaseDebugLibNull:DebugLib.obj
 0001:00000268       DebugPrintLevelEnabled     0000000000000528 f   BaseDebugLibNull:DebugLib.obj
 0001:00000268       DebugPrintEnabled          0000000000000528 f   BaseDebugLibNull:DebugLib.obj
 0001:0000026c       UefiBootServicesTableLibConstructor 000000000000052c f   UefiBootServicesTableLib:UefiBootServicesTableLib.obj
 0001:00000288       UefiRuntimeServicesTableLibConstructor 0000000000000548 f   UefiRuntimeServicesTableLib:UefiRuntimeServicesTableLib.obj
 0001:00000298       UefiLibConstructor         0000000000000558 f   UefiLib:UefiLib.obj
 0001:0000029c       InternalPrint              000000000000055c f   UefiLib:UefiLibPrint.obj
 0001:00000320       Print                      00000000000005e0 f   UefiLib:UefiLibPrint.obj
 0001:00000350       InternalAllocatePool       0000000000000610 f   UefiMemoryAllocationLib:MemoryAllocationLib.obj
 0001:00000388       BasePrintLibFillBuffer     0000000000000648 f   BasePrintLib:PrintLibInternal.obj
 0001:000003bc       BasePrintLibValueToString  000000000000067c f   BasePrintLib:PrintLibInternal.obj
 0001:0000040c       BasePrintLibSPrintMarker   00000000000006cc f   BasePrintLib:PrintLibInternal.obj
 0001:000010f4       BasePrintLibSPrint         00000000000013b4 f   BasePrintLib:PrintLibInternal.obj
 0001:00001118       ReadUnaligned16            00000000000013d8 f   BaseLib:Unaligned.obj
 0001:00001160       ReadUnaligned32            0000000000001420 f   BaseLib:Unaligned.obj
 0001:000011a8       AsciiStrnLenS              0000000000001468 f   BaseLib:SafeString.obj
 0001:00001214       StrnLenS                   00000000000014d4 f   BaseLib:SafeString.obj
 0001:000012b8       InternalMathDivRemU64x32   0000000000001578 f   BaseLib:Math64.obj
 0001:00001310       DivU64x32Remainder         00000000000015d0 f   BaseLib:DivU64x32Remainder.obj
 0002:00000038       ??_C@_0CD@BDCLIGHD@?$CI?$CIUINTN?$CJ?5String?5?$CG?50x00000001?$CJ?5?$DN?$DN@ 0000000000001678     BaseLib:String.obj
 0002:00000060       ??_C@_0CO@LCDFADJO@d?3?2udk2017?2MdePkg?2Library?2BaseLi@ 00000000000016a0     BaseLib:Unaligned.obj
 0002:00000090       ??_C@_0CP@BEPDJGAB@d?3?2udk2017?2MdePkg?2Library?2BaseLi@ 00000000000016d0     BaseLib:SafeString.obj
 0002:000000c0       ??_C@_0N@KGHEHMDL@Divisor?5?$CB?$DN?50?$AA@ 0000000000001700     BaseLib:DivU64x32.obj
 0002:000000d0       ??_C@_0DH@HGAAFDIA@d?3?2udk2017?2MdePkg?2Library?2BaseLi@ 0000000000001710     BaseLib:DivU64x32Remainder.obj
 0002:00000108       _gUefiDriverRevision       0000000000001748     returnadd:AutoGen.obj
 0002:00000110       ??_C@_0CB@DMEJJJHA@?6ASSERT_EFI_ERROR?5?$CIStatus?5?$DN?5?$CFr?$CJ?6@ 0000000000001750     returnadd:AutoGen.obj
 0002:00000138       ??_C@_0BE@DCHLEIGN@?$CBEFI_ERROR?5?$CIStatus?$CJ?$AA@ 0000000000001778     returnadd:AutoGen.obj
 0002:00000150       ??_C@_0GM@MLGLPOID@d?3?2udk2017?2Build?2AppPkg?2DEBUG_VS@ 0000000000001790     returnadd:AutoGen.obj
 0002:000001c0       ??_C@_1CG@PNEGEHON@?$AAr?$AAe?$AAt?$AAu?$AAr?$AAn?$AA?5?$AAh?$AAe?$AAr?$AAe?$AA?5?$AA?$FL?$AA?$CF?$AAX?$AA?$FN?$AA?5?$AA?6?$AA?$AA@ 0000000000001800     returnadd:returnaddress.obj
 0002:000001e8       ??_C@_0BH@IACGKAP@Buffer?5?$CB?$DN?5?$CI?$CIvoid?5?$CK?$CJ?50?$CJ?$AA@ 0000000000001828     UefiLib:UefiLibPrint.obj
 0002:00000200       ??_C@_07PBILKAFL@Success?$AA@ 0000000000001840     BasePrintLib:PrintLibInternal.obj
 0002:00000208       ??_C@_0BG@CFJMNNJK@Warning?5Unknown?5Glyph?$AA@ 0000000000001848     BasePrintLib:PrintLibInternal.obj
 0002:00000220       ??_C@_0BH@GKKCJEPJ@Warning?5Delete?5Failure?$AA@ 0000000000001860     BasePrintLib:PrintLibInternal.obj
 0002:00000238       ??_C@_0BG@ECIJMOED@Warning?5Write?5Failure?$AA@ 0000000000001878     BasePrintLib:PrintLibInternal.obj
 0002:00000250       ??_C@_0BJ@ODIPDGHB@Warning?5Buffer?5Too?5Small?$AA@ 0000000000001890     BasePrintLib:PrintLibInternal.obj
 0002:00000270       ??_C@_0BD@IFJNJCCO@Warning?5Stale?5Data?$AA@ 00000000000018b0     BasePrintLib:PrintLibInternal.obj
 0002:00000288       ??_C@_0L@PLPBEPPC@Load?5Error?$AA@ 00000000000018c8     BasePrintLib:PrintLibInternal.obj
 0002:00000298       ??_C@_0BC@HOFHKGJN@Invalid?5Parameter?$AA@ 00000000000018d8     BasePrintLib:PrintLibInternal.obj
 0002:000002b0       ??_C@_0M@BEECMOIL@Unsupported?$AA@ 00000000000018f0     BasePrintLib:PrintLibInternal.obj
 0002:000002c0       ??_C@_0BA@FLNMPMCF@Bad?5Buffer?5Size?$AA@ 0000000000001900     BasePrintLib:PrintLibInternal.obj
 0002:000002d0       ??_C@_0BB@EGELJFOB@Buffer?5Too?5Small?$AA@ 0000000000001910     BasePrintLib:PrintLibInternal.obj
 0002:000002e8       ??_C@_09NKFGCIPN@Not?5Ready?$AA@ 0000000000001928     BasePrintLib:PrintLibInternal.obj
 0002:000002f8       ??_C@_0N@HHEABDHO@Device?5Error?$AA@ 0000000000001938     BasePrintLib:PrintLibInternal.obj
 0002:00000308       ??_C@_0BA@LNEDDFNB@Write?5Protected?$AA@ 0000000000001948     BasePrintLib:PrintLibInternal.obj
 0002:00000318       ??_C@_0BB@GOILNEAA@Out?5of?5Resources?$AA@ 0000000000001958     BasePrintLib:PrintLibInternal.obj
 0002:00000330       ??_C@_0P@EIOJGIF@Volume?5Corrupt?$AA@ 0000000000001970     BasePrintLib:PrintLibInternal.obj
 0002:00000340       ??_C@_0M@HDLEPOFA@Volume?5Full?$AA@ 0000000000001980     BasePrintLib:PrintLibInternal.obj
 0002:00000350       ??_C@_08KEGAJDNN@No?5Media?$AA@ 0000000000001990     BasePrintLib:PrintLibInternal.obj
 0002:00000360       ??_C@_0O@JNCJKCCD@Media?5changed?$AA@ 00000000000019a0     BasePrintLib:PrintLibInternal.obj
 0002:00000370       ??_C@_09CFCBFJND@Not?5Found?$AA@ 00000000000019b0     BasePrintLib:PrintLibInternal.obj
 0002:00000380       ??_C@_0O@NFHOBIDO@Access?5Denied?$AA@ 00000000000019c0     BasePrintLib:PrintLibInternal.obj
 0002:00000390       ??_C@_0M@ENKCBFEP@No?5Response?$AA@ 00000000000019d0     BasePrintLib:PrintLibInternal.obj
 0002:000003a0       ??_C@_0L@IFPBNFC@No?5mapping?$AA@ 00000000000019e0     BasePrintLib:PrintLibInternal.obj
 0002:000003b0       ??_C@_08PAFJCNGP@Time?5out?$AA@ 00000000000019f0     BasePrintLib:PrintLibInternal.obj
 0002:000003c0       ??_C@_0M@DCJFAFHJ@Not?5started?$AA@ 0000000000001a00     BasePrintLib:PrintLibInternal.obj
 0002:000003d0       ??_C@_0BA@IGIBFFPH@Already?5started?$AA@ 0000000000001a10     BasePrintLib:PrintLibInternal.obj
 0002:000003e0       ??_C@_07LCKDCBKK@Aborted?$AA@ 0000000000001a20     BasePrintLib:PrintLibInternal.obj
 0002:000003e8       ??_C@_0L@LKIFCMNO@ICMP?5Error?$AA@ 0000000000001a28     BasePrintLib:PrintLibInternal.obj
 0002:000003f8       ??_C@_0L@DJKNJKHM@TFTP?5Error?$AA@ 0000000000001a38     BasePrintLib:PrintLibInternal.obj
 0002:00000408       ??_C@_0P@NCJHBCLM@Protocol?5Error?$AA@ 0000000000001a48     BasePrintLib:PrintLibInternal.obj
 0002:00000418       ??_C@_0BF@EHOBGFMI@Incompatible?5Version?$AA@ 0000000000001a58     BasePrintLib:PrintLibInternal.obj
 0002:00000430       ??_C@_0BD@KHMPCIOG@Security?5Violation?$AA@ 0000000000001a70     BasePrintLib:PrintLibInternal.obj
 0002:00000448       ??_C@_09BOMAGJEG@CRC?5Error?$AA@ 0000000000001a88     BasePrintLib:PrintLibInternal.obj
 0002:00000458       ??_C@_0N@JEJDHPO@End?5of?5Media?$AA@ 0000000000001a98     BasePrintLib:PrintLibInternal.obj
 0002:00000468       ??_C@_0O@NMJOLAMF@Reserved?5?$CI29?$CJ?$AA@ 0000000000001aa8     BasePrintLib:PrintLibInternal.obj
 0002:00000478       ??_C@_0O@GLPDOMCP@Reserved?5?$CI30?$CJ?$AA@ 0000000000001ab8     BasePrintLib:PrintLibInternal.obj
 0002:00000488       ??_C@_0M@FKGOBENP@End?5of?5File?$AA@ 0000000000001ac8     BasePrintLib:PrintLibInternal.obj
 0002:00000498       ??_C@_0BB@KFJAMCOC@Invalid?5Language?$AA@ 0000000000001ad8     BasePrintLib:PrintLibInternal.obj
 0002:000004b0       ??_C@_0BB@MFGDFIJM@Compromised?5Data?$AA@ 0000000000001af0     BasePrintLib:PrintLibInternal.obj
 0002:000004c8       ??_C@_0O@MLOLIMFM@?$DMnull?5string?$DO?$AA@ 0000000000001b08     BasePrintLib:PrintLibInternal.obj
 0002:000004d8       ??_C@_0M@BJJDNPHK@?$DMnull?5guid?$DO?$AA@ 0000000000001b18     BasePrintLib:PrintLibInternal.obj
 0002:000004e8       ??_C@_0DB@PMLHLBMO@?$CF08x?9?$CF04x?9?$CF04x?9?$CF02x?$CF02x?9?$CF02x?$CF02x@ 0000000000001b28     BasePrintLib:PrintLibInternal.obj
 0002:00000520       ??_C@_0M@LHGBCIKM@?$DMnull?5time?$DO?$AA@ 0000000000001b60     BasePrintLib:PrintLibInternal.obj
 0002:00000530       ??_C@_0BK@FCPKCIDD@?$CF02d?1?$CF02d?1?$CF04d?5?5?$CF02d?3?$CF02d?$AA@ 0000000000001b70     BasePrintLib:PrintLibInternal.obj
 0002:0000054c       ??_C@_04JIMNDDED@?$CF08X?$AA@ 0000000000001b8c     BasePrintLib:PrintLibInternal.obj
 0002:00000554       ??_C@_02PCIJFNDE@?$AN?6?$AA@ 0000000000001b94     BasePrintLib:PrintLibInternal.obj
 0002:00000558       ??_C@_01LIIJDEN@?$AN?$AA@  0000000000001b98     BasePrintLib:PrintLibInternal.obj
 0002:00000560       mHexStr                    0000000000001ba0     BasePrintLib:PrintLibInternal.obj
 0002:00000570       mStatusString              0000000000001bb0     BasePrintLib:PrintLibInternal.obj
 0003:00000000       gImageHandle               0000000000001da0     UefiBootServicesTableLib:UefiBootServicesTableLib.obj
 0003:00000008       gST                        0000000000001da8     UefiBootServicesTableLib:UefiBootServicesTableLib.obj
 0003:00000010       gBS                        0000000000001db0     UefiBootServicesTableLib:UefiBootServicesTableLib.obj
 0003:00000018       gRT                        0000000000001db8     UefiRuntimeServicesTableLib:UefiRuntimeServicesTableLib.obj

 entry point at        0001:00000000

 Static symbols

 0004:00000000       $pdata$_ModuleEntryPoint   0000000000001dc0     * CIL library *:* CIL module *
 0004:0000000c       $pdata$ProcessLibraryConstructorList 0000000000001dcc     * CIL library *:* CIL module *
 0004:00000018       $pdata$ProcessModuleEntryPointList 0000000000001dd8     * CIL library *:* CIL module *
 0004:00000024       $pdata$UefiMain            0000000000001de4     * CIL library *:* CIL module *
 0004:00000030       $pdata$InternalPrint       0000000000001df0     * CIL library *:* CIL module *
 0004:0000003c       $pdata$Print               0000000000001dfc     * CIL library *:* CIL module *
 0004:00000048       $pdata$InternalAllocatePool 0000000000001e08     * CIL library *:* CIL module *
 0004:00000054       $pdata$BasePrintLibValueToString 0000000000001e14     * CIL library *:* CIL module *
 0004:00000060       $pdata$BasePrintLibSPrintMarker 0000000000001e20     * CIL library *:* CIL module *
 0004:0000006c       $pdata$BasePrintLibSPrint  0000000000001e2c     * CIL library *:* CIL module *
 0004:00000078       $pdata$ReadUnaligned16     0000000000001e38     BaseLib:Unaligned.obj
 0004:00000084       $pdata$ReadUnaligned32     0000000000001e44     BaseLib:Unaligned.obj
 0004:00000090       $pdata$AsciiStrnLenS       0000000000001e50     BaseLib:SafeString.obj
 0004:0000009c       $pdata$StrnLenS            0000000000001e5c     BaseLib:SafeString.obj
 0004:000000a8       $pdata$InternalMathDivRemU64x32 0000000000001e68     BaseLib:Math64.obj
 0004:000000b4       $pdata$DivU64x32Remainder  0000000000001e74     BaseLib:DivU64x32Remainder.obj
 0005:00000000       $unwind$_ModuleEntryPoint  0000000000001e80     * CIL library *:* CIL module *
 0005:00000010       $unwind$ProcessLibraryConstructorList 0000000000001e90     * CIL library *:* CIL module *
 0005:00000010       $unwind$StrnLenS           0000000000001e90     * CIL library *:* CIL module *
 0005:00000018       $unwind$ProcessModuleEntryPointList 0000000000001e98     * CIL library *:* CIL module *
 0005:00000018       $unwind$UefiMain           0000000000001e98     * CIL library *:* CIL module *
 0005:00000020       $unwind$InternalPrint      0000000000001ea0     * CIL library *:* CIL module *
 0005:00000034       $unwind$Print              0000000000001eb4     * CIL library *:* CIL module *
 0005:0000003c       $unwind$InternalAllocatePool 0000000000001ebc     * CIL library *:* CIL module *
 0005:0000003c       $unwind$ReadUnaligned16    0000000000001ebc     * CIL library *:* CIL module *
 0005:0000003c       $unwind$ReadUnaligned32    0000000000001ebc     * CIL library *:* CIL module *
 0005:00000044       $unwind$BasePrintLibValueToString 0000000000001ec4     * CIL library *:* CIL module *
 0005:00000050       $unwind$BasePrintLibSPrintMarker 0000000000001ed0     * CIL library *:* CIL module *
 0005:0000006c       $unwind$BasePrintLibSPrint 0000000000001eec     * CIL library *:* CIL module *
 0005:00000074       $unwind$AsciiStrnLenS      0000000000001ef4     BaseLib:SafeString.obj
 0005:0000007c       $unwind$InternalMathDivRemU64x32 0000000000001efc     BaseLib:Math64.obj
 0005:00000084       $unwind$DivU64x32Remainder 0000000000001f04     BaseLib:DivU64x32Remainder.obj
